:1000000002044D0207ACFFFFFFFFFF0207BEFFFF28
:10001000FFFFFF0207B6FFFFFFFFFF0208CDFFFF54
:10002000FFFFFF02044DFFFFFFFFFF02044DFFFF34
:10003000FFFFFFFFFFFFFFFFFFFFFFFFFFFFFFFFD0
:10004000FFFFFF02044DFFFFFFFFFF02044DFFFF14
:10005000FFFFFF02044DFFFFFFFFFF02044DFFFF04
:10006000FFFFFF02044DFFFFFFFFFF02044DC290A0
:1000700075831E758200D582FDD583FA7420120126
:1000800036748012013675830F758200D582FDD5D6
:1000900083FA74201201367480120136758301755B
:1000A0008233D582FDD583FA74061200BD740C121A
:1000B00000BD74141200BD22D290C29022C0E01282
:1000C0000104C0E054F0120136D0E0C454F0120133
:1000D00036D0E022C0E0740180E5C0E0740280DF29
:1000E000C0E0748080D9C0E074C080D3C0E07418D0
:1000F00080CDC0E0741C80C7C0E0740780C1C0E040
:10010000448080BBC0E05390FA4390F2D290E590D7
:10011000C290D290C29020E7F3D0E022C0E0310438
:10012000C0E054F04404120136D0E0C454F044045A
:10013000120136D0E0224408529054F7429001B8A0
:10014000C0E0742080D811E0C0E01581D083D08257
:10015000058105810581740093B40010A3158115F4
:10016000811581C082C0830581D0E022B41F004088
:1001700002311CB40206A374009311FEA380D711B0
:10018000E680C5540F04832230313233343536379C
:1001900038394142434445463183311C22C0D0C0E6
:1001A000E0C43198D0E03198D0D022C0E011E08096
:1001B00004C0E011E6E8319D3140E9319D3140EA6B
:1001C000319D3140EB319D3140EC319D3140ED317D
:1001D0009D3140EE319D3140EF319DD0E022400213
:1001E0008009C0E07431311CD0E022C0E07430805E
:1001F000F5C0E0C0D011E08006C0E0C0D011E6E557
:10020000D0319D3140D0D0D0E0C0E0319D3140E5CB
:1002100081319D3140C082C083E583319D3140E50D
:1002200082319DD083D082D0E02231AB80CB512A65
:1002300080FE7583008583827814D582FDD583FA8C
:10024000D8F812025F11D422C0E0780875F008A433
:10025000444011BD740093311CA3D8F8D0E022C0F3
:10026000E0C082C08374007908900278514804D9B4
:10027000FBD083D082D0E0220204081F08040200D1
:100280000804021F0204080000110A040A110000F9
:100290000000010214080000060A0200060909060F
:1002A0001F1F1F1F1F1F1F1F1F1F1F1F1F1F1F1F5E
:1002B0001F1F1F1F1F1F1F1FC083C0828583308504
:1002C0008231D082D08322C0E053D0FF43D0185176
:1002D000B8F5321202F01202DF53D0E7D0E0225319
:1002E000D0FF43D01851B81203AEE53253D0E72205
:1002F00012034B74057F0412033FE5307F031203A2
:100300003F74007F0112033F12036DE5317F081235
:10031000033F12036DE5327F0812033F12036D1293
:10032000035E120326227B40DB02800F12034B7414
:10033000857F0812033F12036D40ED12035E22C257
:10034000A1C2A11392A0D2A1DFF7220000D2A10086
:1003500000D2A00000C2A00000C2A1000022000044
:10036000C2A00000D2A10000D2A000002200000024
:1003700000C2A10000D2A000000000D2A100000035
:10038000000000A2A0C2A10000220000C2A1000043
:10039000C2A000000000D2A10000C2A10000D2A0B3
:1003A000000022D2A00000D2A10000C2A122714B05
:1003B00074057F04713FE5307F03713F74007F0156
:1003C000713F716DE5317F08713F716D714B74053F
:1003D0007F04713FE5307F03713F74017F01713FFE
:1003E000716D7F08D2A10000A2A0C2A1E53213F571
:1003F00032DFF171A3715E715E22E5A054F0B4F0BA
:10040000047400C322E5A054F060EFC4900412937A
:10041000801000000006000A080400070903050216
:100420000100D322D22371FA50FAC083C0827583AF
:1004300008758200D582FDD583FAD082D08371FA07
:1004400050E2C0E071FA40FCD0E0C22322121AF45C
:100450007800E4F608B880FB75A80075D0007581B7
:1004600076116E116E11D411DA3146444C344A4182
:100470004C2062792053574A5A445A00317F205603
:10048000657273696F6E20312E35312E3033200046
:100490005132116E116E11D411DA3146737032730C
:1004A000776A2E73702D7172702E706C00317F73AD
:1004B000703273776A406F702E706C20367820002F
:1004C0005132755A1871FAB4034A314802004B612F
:1004D000736F77616E696520454550524F4D00310D
:1004E00048024050757363206B6C617769737A00C2
:1004F000912431480240706F637A656B616A2032E3
:10050000302073656B2E0090000074FF51C7A3E587
:1005100083B408F6121714E5637004D2088002C28F
:1005200008E5627002D293E554600312191A71FA59
:10053000200803020699B4010B201905120B16803E
:10054000031208F3B4020B2019051212868003125D
:10055000095AB4030B20190512138D8003120A1BCC
:10056000B4040E2019051214F180061214F10206CB
:10057000992019FAB4063D3148024020202020205D
:10058000205041534D4F20203E203E009124121810
:10059000F5055EC0E0E55EB40B03755E00E55E90B8
:1005A00007FF51C712164A121BF911D4121DAB12C4
:1005B0001E10D0E0B407223148024D524954009138
:1005C000243148024D20202000E55DC0E0755D0328
:1005D00074031215C7D0E0F55DB4053D3148024003
:1005E0003C203C20205041534D4F202020202020F3
:1005F0000091241218F5155EC0E0E55EB4FF0375A6
:100600005E0AE55E9007FF51C712164A121BF911E8
:10061000D4121DAB121E10D0E0B408233148024D95
:1006200053504C0091243148024D2020202000E5F9
:100630005DC0E0755D0374021215C0D0E0F55DB4D5
:10064000093A3148020C4D4F44450091243148028B
:100650000C2020202000C0E0E57404B40401E4F57F
:1006600074E5805530F5F0E574C445F0F580E5A0FB
:1006700054F0440FF470F7121E10D0E0B40A1A318F
:1006800048024056464F207A61706973616E65007A
:100690009124C0E01218F5D0E01207D130190302FE
:1006A0000725301B0F20A30612073A020725120761
:1006B0008502072520091230A20530A30280051209
:1006C000073A8061120785805C12078D300D1A127F
:1006D000073AC20F120798120785120798856163BF
:1006E000856062D28CD28EC20D12078D300E36120A
:1006F000073AC20FE572B40402D20F120798B4038E
:1007000002D20F120798B40202D20F120798B40156
:1007100002D20F120785120798856163856062D245
:100720008CD28EC20E300810121DAB121E10C28C5D
:10073000C28E438701438720A117301B2F308609C3
:10074000C286C293C208121C7620A210201C2975F2
:100750005F05201F03755F03D21C8013301C1975C1
:100760005F03201F03755F05C21C8003308609C22A
:1007700086C293C208121C76856163856062D28C42
:10078000D28ED20322D286121C76C2032220A2026B
:10079000D20D20A302D20E2253A8FBAA71300F0261
:1007A000F18D7BFFDBFEDAF543A8042230B40405AB
:1007B00054800215543232758CD8758AF022C0E00C
:1007C000F1B7E56360021563E56260021562D0E08F
:1007D00032E5805430B573028007D21EF573121BC8
:1007E000F9301D03020851E580540FB55E028061A7
:1007F000B40F3611D4E580540FB40F2D31480200E8
:10080000205A414C4F5A20205A574F524B492020D2
:1008100000120148024020205A4D49414E592050B3
:1008200041534D2020200080CC1200D47F007E0058
:10083000DEFEDFFAE580540FB55E0280141218F573
:10084000F55E12164A121BF91200D4121DAB121ECD
:1008500010744F1200FE7420200802744212011C12
:10086000744E1200FE7420209302744E02011CFB91
:100870001DFC17FCBEFD35FD8EFDD4FE06C083C0F9
:1008800082C0E0E55FB4000590086F8030B40105D8
:100890009008718028B402059008738020B4030585
:1008A0009008758018B404059008778010B4050589
:1008B0009008798008B4060590087B8000E493F5E1
:1008C0008D740193F58BD0E0D082D08322C0E011EB
:1008D0007D300304B2878004D287C28ED0E032E537
:1008E0005420E7070303543FC38007F40403035471
:1008F0003FD3221200D412014802004B726F6B3AB0
:1009000000C0E0E559B40012755903C2061201484F
:100910000240313020487A00803BB40312755909F7
:10092000C206120148024031206B487A008026B48A
:10093000091475590AC206120148024031303020AC
:100940006B487A00800F755900C2061201480240B8
:100950003120487A00D0E00204241200D412014869
:100960000200576F62756C6F77616E696520422D6A
:100970003E4100120148024053746F70203D2061D7
:100980006E796B6579001204241209EF50157843D3
:10099000794F121B3E78477943121B3E784F7947B7
:1009A000121B3E7847794F121B3EC2A2C2A3120A05
:1009B00013D2A2D2A3C20A121BF91209FD784A79F6
:1009C0006C121F38121BF91209EF500E1209FDC2EA
:1009D000A2C2A3120A13D2A2D2A31203FA50DE12A9
:1009E0000424120A131200D412185B755400227FDB
:1009F000047846794AC3E6971819DFFA22B2212013
:100A00002109120148024E58008007120148024E87
:100A10004F0022784F7947121B3E22756D00756E8C
:100A200000756F007570001200D412014802005367
:100A30006B6F6B20776F62756C6F77616E696100A9
:100A40001201480249487A00120A92120424E5541D
:100A50006031C0E0755400757001756F001203FAC3
:100A6000B40106757010756F00B4020675700075DC
:100A70006F01786C7970D0E020E705121F38800391
:100A8000121F44120A921203FAB404C275540002EF
:100A9000042474401200FE7F047869E612019D0868
:100AA000DFF922120148020020204B4F4E464947F1
:100AB000555241434A4120200022120148020020A1
:100AC000205A4D49414E41205041534D4120200074
:100AD0002212014802003C3C202020204D454E556A
:100AE000202020203E3E002212014802002020202B
:100AF0002046554E4B434A41202020202000221200
:100B000001480200202020555354415749454E4981
:100B1000452020200022C2051200D4E55AB4001559
:100B200051A31201480240506F737265646E69658B
:100B30006A20435700B4011651A3120148024050E5
:100B40006F737265646E69656A204C534200B4022B
:100B50001651A31201480240506F737265646E69AA
:100B6000656A2055534200B4031751A3120148028D
:100B7000405472796220706F737265646E69656A41
:100B800000B4041851A31201480240437A617375FE
:100B900020426C6F6B6F77616E696100B40518510C
:100BA000A31201480240437A61737520706F647428
:100BB0002E206E61642E00B4061451FF120148020B
:100BC0004054656D7061204B6C75637A6100B407A9
:100BD0002D51E812014802404B6C75637A2043574F
:100BE0000020090E120148024A7A616C61637A00A2
:100BF000800C120148024A77796C61637A00B4086C
:100C00001651FF120148024050616D696563692009
:100C10006B726F706B6900B4093351A31201480203
:100C2000404E61642E0020001212014802444357D6
:100C3000207A20706F73722E0080121201480244D5
:100C400043572062657A20706F73722E00B40A2BAE
:100C500051A312014802404772616E6963652050DA
:100C600041534D00201A0B120148024D7A616C006D
:100C70008009120148024D77796C00B40B2D51FFA9
:100C80001201480240547279622046534B00201BE7
:100C90000E12014802497A616C61637A00800C127D
:100CA0000148024977796C61637A00B40C491201FA
:100CB00048020050525A454C41435A4E494B20502D
:100CC00041534D00201D1B1201480240202020539B
:100CD0007465726F77616E69652020200043800F14
:100CE0008015120148024020202020204F64637AA2
:100CF00079742020202000B40D1551BA1201480249
:100D0000403136306D2020312C38204D487A00B4E7
:100D10000E1551BA12014802402038306D202033A0
:100D20002C35204D487A00B40F1551BA12014802F3
:100D3000402034306D2020202037204D487A00B4E8
:100D4000101651BA12014802402033306D20203174
:100D5000302C35204D487A00B4111451BA12014894
:100D600002402032306D20203134204D487A00B4CA
:100D7000121451BA12014802402031376D2020313F
:100D800038204D487A00B4131451BA120148024079
:100D90002031356D20203231204D487A00B41414B2
:100DA00051BA12014802402031326D2020323420E5
:100DB0004D487A00B4151451BA120148024020314E
:100DC000306D20203238204D487A00B4161651BAC2
:100DD00012014802405472737620366D203530205F
:100DE0004D487A00B4171751BA12014802405472A4
:100DF000737620326D20313434204D487A00B41897
:100E00001851D112014802402020202057594A533E
:100E100043494520202020200011DF6034D2057591
:100E200054004016055AE55A201D07B40D047418E5
:100E3000F55AB41903755A008014155AE55A201D45
:100E400007B41704740CF55AB4FF03755A1812004E
:100E5000D41203FA5002611B200500E55AB40016B3
:100E600090000B78651218EA120F9290000B7865CB
:100E70001218DF020F8DB4011690000F786512185A
:100E8000EA120F9290000F78651218DF020F8DB4EE
:100E9000021690001378651218EA120F9290001350
:100EA00078651218DF020F8DB40306121034020F9A
:100EB0008DB4040DE5611211ABF56112189A020FA1
:100EC0008DB4050DE5601211ABF5601218AB020F81
:100ED0008DB4060FE571F412118BF4F571121889B7
:100EE000020F8DB40715B2099000071202DFA209A4
:100EF00092E79000071202C7020F8DB40810E57246
:100F000012120BF5729000061202C7020F8DB4097F
:100F100015B2009000071202DFA20092E6900007CF
:100F20001202C7020F8DB40A15B21A9000071202FE
:100F3000DFA21A92E59000071202C7020F8DB40BD0
:100F400015B21B201B08121807755F038002C20927
:100F500012185B020F8DB40C1AB21D90000712021A
:100F6000DFA21D92E49000071202C7201D034380F8
:100F70000F801AB418028015C0E01218F5D0E0C333
:100F8000940DF55E9007FF1202C712164AD21E0298
:100F900016037569401200D4744A1200FE740012E0
:100FA000011C0412011C0412011C0412011CE5693D
:100FB0001200FE742312011C74001200FE78657F7B
:100FC00004E612019D08DFF91203FA502E120424E0
:100FD000B4010A1569E569B43F03756947B4020AAB
:100FE0000569E569B44803756940B40306D0E0D0EB
:100FF000E0809AB40402803B1200D411DF603140DB
:101000002C1200D4E569135012541F2465F806E62B
:10101000540FB40A04E654F0F68012541F2465F805
:10102000E62410F654F0B4A004E6540FF67554000C
:10103000020F98227569401200D49000021202DF5C
:10104000F565A31202DFF566744A1200FE74001201
:10105000011C0412011C740412011C740312011CF3
:1010600074001200FEE565A2E71201DEA2E612019D
:10107000DEA2E51201DEA2E41201DEA2E31201DE2D
:10108000A2E21201DEA2E11201DEA2E01201DEE51F
:1010900066A2E71201DEE5691200FE742312011C4C
:1010A0001203FA4003021150120424B4010A156914
:1010B000E569B43F03756948B4020A0569E569B496
:1010C0004903756940B40370E569B44009E565B248
:1010D000E7F56502114DB44109E565B2E6F5650233
:1010E000114DB44209E565B2E5F56502114DB44311
:1010F00009E565B2E4F56502114DB44409E565B250
:10110000E3F56502114DB44509E565B2E2F5650206
:10111000114DB44609E565B2E1F56502114DB447DC
:1011200009E565B2E0F56502114DB44809E566B21E
:10113000E7F56602114D8018B40412900002E565CF
:101140001202C7900003E5661202C780051200D4A0
:101150000148E565A2E79210A2E69211A2E592127B
:10116000A2E49213A2E39214A2E29215A2E19216D3
:10117000A2E09217E566A2E79218229000021202FE
:10118000DFF565A31202DFF56680C7F569755400C7
:101190001200D41201480200537A79626B3A20207F
:1011A00020207A6E616B6F7700801EF569755400A0
:1011B0001200D4120148020054696D65723A202071
:1011C000202030206D53656B00744A1200FE7403BA
:1011D00012011C12011C12011C12011CE569121AD9
:1011E0000474061200FEE565C224121A151203FAF1
:1011F0004011E554600BF5F0E56925F0F56975548B
:101200000080C61203FA40FBE56922F569755400B7
:101210001200D4120148020050616D6965633A0002
:10122000744A1200FE740312011C12011C12011CEC
:1012300012011CE569121A04740A1200FEE565C267
:1012400024121A151203FA4020E554601A20E70A06
:10125000E56904B4050274008008E56914B4FF026E
:101260007404F56975540080B71203FA40FBE56910
:101270002212014802004B726F6B207374726F6A06
:10128000656E69610022C2051200D4E55BB4000EF0
:101290005171120148024020203120487A00B401E7
:1012A0000E5171120148024020203220487A00B4C9
:1012B000020E5171120148024020203520487A0068
:1012C000B4030E5171120148024020313020487A97
:1012D00000B4040E517112014802402032302048FF
:1012E0007A00B4050E5171120148024020353020B9
:1012F000487A00B4060F5171120148024020313083
:101300003020487A001208DF6020D2057554004072
:101310000C055BE55BB40703755B00800A155BE5B4
:101320005BB4FF03755B061200D41203FA5002414E
:101330008B200513E55920060424038003C394037E
:10134000B206F559021351E55B855B59121881C24B
:101350000602160312014802005A61706973207078
:10136000616D69656369001201480240506F7A79C6
:10137000636A613A001213F01202DF04B40A0274C5
:1013800000C0E074491200FED0E002019D1200D4BA
:10139000755C00E55CB4000471548015B40B0F1249
:1013A0000148020057594A5343494500800312142B
:1013B000591208DF601E755400400C055CE55CB4F2
:1013C0000C03755C00800A155CE55CB4FF03755C7A
:1013D0000B1200D41203FA500280B8E55CB4000589
:1013E0001214398008B40B02800312149D021603F4
:1013F000C0E0E55EB40003900083B401039000DF19
:10140000B4020390013BB40303900197B40403902A
:1014100001F3B4050390024FB406039002ABB40786
:1014200003900307B40803900363B409039003BF58
:10143000B40A0390041BD0E02271F01202DF04B45E
:101440000A00400274001202C71214CC78437E08CE
:10145000E61202C708A3DEF822C0E014C0E01201C1
:1014600048020C503A00D0E0C0E012019DD0E0717B
:10147000F01214CC7E0878691202DFF608A3DEF8B9
:1014800074021200FE7869121D8F121DE67442125A
:1014900000FE786D121D8F121DE6D0E0221471F04F
:1014A0001214CC78657E081202DFF608A3DEF87805
:1014B00068301A0C121AB340127868121A6F400B77
:1014C000786579437F08121B40C20C2275F009A48D
:1014D000A32582F582E5F03583F5832212014802C7
:1014E00000437A6573746F746C69776F73633A0045
:1014F00022C2051200D491DC301B18200515120100
:1015000048024046534B206F6477726F746E6500DB
:1015100002157CE55DB40010120148024056464FAA
:10152000202041202F204200B40110120148024027
:1015300056464F202041203D204200B4020B1201AC
:1015400048024053706C697400B4030912014802E8
:101550004052697400B4041212014802405374727C
:101560006F6A656E696520545800B4050F12014812
:1015700002405A617069732056464F001208DF60BE
:1015800020D205755400400C055DE55DB406037579
:101590005D00800A155DE55DB4FF03755D05120011
:1015A000D41203FA500281F6301B08200505B21F41
:1015B000021603E55DB40002B20AB401031216126A
:1015C000B40204C20CB20BB40312200C0B1216129C
:1015D000C20AC20BD20C8004D20AC20CB404191283
:1015E000073A1204241207851203FA40FB7FFFDF3B
:1015F000FE1203FA40F2800BB405051218F58003C1
:10160000B40600755400121BF91200D4121DAB026F
:101610001E10200A067847794380047843794702F0
:101620001B3E01815000035600000703000010110B
:1016300060001406000018096000210600002490D4
:1016400060002806000010000000B40B11D219E45D
:101650007865F608B871FB755900C2068002C21998
:101660007F087843201934300131E55E301D0BC00E
:10167000E05380F04280D0E0800343800F75F00992
:10168000A42420F5827583001202DFF608A3DFF898
:10169000121A6D4006121AB1400122E55EB400052F
:1016A0009016228059B401059016268051B4020587
:1016B00090162A8049B4030590162E8041B4040583
:1016C0009016328039B405059016368031B406057F
:1016D00090163A8029B4070590163E8021B408057B
:1016E0009016428019B409059016428011B40A057B
:1016F0009016428009B40B059016468001227F04A3
:101700007843C082C083121CF0D083D0827F0478DB
:1017100047021CF053890043891143B8081207B7E8
:1017200012087DD28EC203755F0343A88FD288C290
:1017300006C20BC20CC21BC21FD208D20AD21E1292
:1017400018BC20020302177D12185B317B12187639
:101750001218A21218B31218919000071202DFA2F9
:10176000E79209A2E69200A2E5921AA2E4921D1263
:1017700018229000061202DFF5720217EEE47F04D1
:10178000784FF6DFFD7559017561647560327571CA
:1017900080757204C209C200D21A7565FF7566FFB2
:1017A0001218322001030217EE90000B784F121826
:1017B000DF90000F784F1218DF900013784F121847
:1017C000DF12188112189A1218AB121889E572905C
:1017D00000061202C7A20992E7A20092E6A21A929C
:1017E000E5A21D92E49000071202C7121812301DE4
:1017F000089007FF1202DFF55ED14A121BF9121C96
:1018000076121DAB021E109000071202DFA2E792B3
:101810000922E5659000021202C7E5669000030206
:1018200002C79000021202DFF5659000031202DF8A
:10183000F566E565A2E79210A2E69211A2E5921282
:10184000A2E49213A2E39214A2E29215A2E19216EC
:10185000A2E09217E566A2E7921822784F90000B5B
:10186000201B10E5805430B4200390000FB4100307
:101870009000130218EA9000041202DFF559F55B9C
:1018800022900004E5590202C7900008E5710202A7
:10189000C79000081202DFF5712290000AE561028C
:1018A00002C790000A1202DFF56122900009E5608C
:1018B0000202C79000091202DFF5602290000012B8
:1018C00002DFB40104D2028010C20274011202C706
:1018D0009000001202DFB40103D20122C201227F74
:1018E00004E61202C708A3DFF8227F041202DFF623
:1018F00008A3DFF82220191FC0E0E55E75F009A4F7
:1019000024207F087843F582758300E61202C70819
:10191000A3DFF8D0E0800211762275540020190C64
:10192000201B092008063009030219D920080302E8
:101930001A03755500755600755700755800C0E0BC
:10194000E559B400057558018042B4010375580289
:10195000B40203755805B4030375580AB40403753B
:101960005820B40503755850B40603755701B407E1
:1019700003755702B40803755705B409037557106A
:10198000B40A03755610B40B03755501D0E020E777
:1019900020FC121A5D7958121F38201910301A0DC8
:1019A000121AB15008121A5D7958121F44DCE380F4
:1019B00020F404FC121A5D7958121F4420191030CB
:1019C0001A0D121A6D5008121A5D7958121F38DC60
:1019D000E3121BF9121DAB802AF4042571F5711274
:1019E00000D412014802004B6C75637A3A00E5712D
:1019F000F4121A0474071200FEE565C224121A15C7
:101A00008561632275F06484F565740AC5F084C449
:101A100025F0F56622E565C0E0C4120183B4300507
:101A20001201408005D22412011CD0E01201832053
:101A30002408B430051201408005D22412011CE5AF
:101A400066C0E0C4120183202408B43005120140AE
:101A5000800312011CD0E012018302011C78462091
:101A60000A02784A227843200A02784722515D7F91
:101A700004901A85E55E23232403FEC3EE93961893
:101A80001EDFF9B32201800000034900000699001F
:101A9000001009000013990000180670002099003A
:101AA000002488000027990000279900002799004A
:101AB00000515D7F04901AC8E55E23232403FEC312
:101AC000EE9396181EDFF922020000000381000049
:101AD000072100001016000014360000181700003F
:101AE0002146000025000000297100002971000036
:101AF00030010000C2B7C2B5C2B67400121CDEC20B
:101B0000B5D2B5C2B57400121CDEC2B5D2B5C2B52D
:101B10007400121CDEC2B5D2B5C2B57400121CDE50
:101B2000C2B5D2B5C2B57400121CDEC2B5D2B5C200
:101B3000B52278438006784780025165794B7F044F
:101B4000E6F70809DFFA22E55EB400093010030267
:101B50001BBF021BC6B40109301103021BBF021BCD
:101B6000C6B40209301203021BBF021BC6B403092C
:101B7000301303021BBF021BC6B404093014030256
:101B80001BBF021BC6B40509301503021BBF021B95
:101B9000C6B40609301603021BBF021BC6B40709F0
:101BA000301703021BBF021BC6B408028008B40929
:101BB000028003B40A09301803021BBF021BC67857
:101BC0004E7952021F38784E7952021F44000001AC
:101BD00070901BCD7F047865121CF0784E796802F6
:101BE0001F38121CBA793B800C121CBA793380055D
:101BF000121CBA79377865613EC2AF301E04115BA2
:101C0000C21E301907713A71E9021C76300C1C7142
:101C100036714771E971323020033000027147712B
:101C2000F0301B0471D171E2021C76300B20713A46
:101C3000714771E9B20A713A3020033000027147EE
:101C400071F0301B0471D171E2B20A021C76713A54
:101C5000302003300002714771F03020033000065D
:101C600078657933713E301B0471D171E220000632
:101C7000713A714771E9C2AF201926301B1C2086CA
:101C80001520A205301F078009301F068000783E0E
:101C90008011783A800D78368009208604783A8061
:101CA0000278367E04E6121CDE18DEF97401121C7E
:101CB000DEC2B5D2B5C2B5D2AF2275650075660079
:101CC000756700756800121D2C121D36121D3F121B
:101CD0001D49121D52121D5C121D65021D6F7D08EB
:101CE000135004D2B78002C2B7D2B6C2B6DDF12219
:101CF000C0E0E493F6A308DFF9D0E022783F7F0448
:101D000080EE540FFE78427F047553008EF0E6A4F7
:101D1000255385F05350020553F618DFEF786879A4
:101D2000427F04C3E736F61819DFF922901F63914A
:101D3000FCE54BC480CC901F6791FCE54B80C390C1
:101D40001F6B91FCE54CC480B9901F6F91FCE54C72
:101D500080B0901F7391FCE54DC480A6901F7791D1
:101D6000FCE54D809D901F7B91FCE54EC4809390D7
:101D70001F7F91FCE54E808A540F4430BF0705B4A5
:101D80003002742002011C0000002200000016E551
:101D90005EB40905901D878006B40A0E901D8BE87D
:101DA0002403F97868121F26786522200B0D200C79
:101DB0000A12014802004120008008120148020076
:101DC0002020007843B18F121DE6200B0D200C0A55
:101DD00012014802404220008008120148024020BF
:101DE00020007847B18F7F07BF0505742C12011CB6
:101DF000E6C0E0C4B1781FBF0006D0E0B178800F24
:101E0000BF0205742E12011CD0E0B17808DFD92280
:101E100030060F740B200A02744B1200FE742A1253
:101E2000011C301B1CC220301F0B120148020D4642
:101E30005352008009120148020D46534B00021E06
:101E40008BE5805430B40010120148020D43572036
:101E5000002020041107D220B4100D120148020DF9
:101E600055534200C220C209B4200D120148020D90
:101E70004C534200C220C209B43010120148020D76
:101E800043576E002020041107D220300B2B744DD5
:101E90001200FE745312011C200A101201480200A5
:101EA0004E0012014802404F00800E12014802000D
:101EB0004F0012014802404E00300C18744D1200C1
:101EC000FE745212011C12014802004E0012014819
:101ED00002404F00200A0912014802413E008007DB
:101EE00012014802013E0020190122E559B4000BFD
:101EF000120148024C2031487A0022B4030B12012F
:101F000048024C3130487A0022B4090B12014802D1
:101F10004C316B487A0022B40A0B120148024C3152
:101F200030306B0022227A04C39222E493A222373B
:101F3000D4F6A31819DAF2227A04C3E637D4F618D5
:101F400019DAF8227A04C3E69710D70730D60C9432
:101F500006800830D60294069460D3F61819DAE7A2
:101F60002200FF0E38E38E016C16C1002468AD001C
:101F700003A41100005D3500000952000000EF00CD
:051F8000000018FF0045
:00000001FF
